:0200000480007A
:10000000B72F0000938F0F8073900F3015A8130047
:100010000000130000001300000013000000130094
:100020000000130000001300000013000000130084
:100030000000130000001300000013000000010086
:10004000970200009382020C73905230814001416C
:100050008141014281420143814301448144014580
:100060008145014681460147814701488148014950
:100070008149014A814A014B814B014C814C014D20
:10008000814D014E814E014F814F971102009381A6
:1000900061B5170502001305E536979503009385B2
:1000A000A56B01461122170502001305E5329705DD
:1000B00002009385E5320146C52817A50300130504
:1000C000E56997B503009385256937B6ABAB130691
:1000D000B6BAD92817B1030013014168EF40D01F09
:1000E000860293D21200F512638802008242110147
:1000F0006F00001073002030824211017300203025
:10010000711116C0F3222034E3CC02FC82421101AB
:10011000130141F806C20AC40EC612C816CA1ACC88
:100120001ECE22D026D22AD42ED632D836DA3ADCC7
:100130003EDEC2C0C6C2CAC4CEC6D2C8D6CADACC97
:10014000DECEE2D0E6D2EAD4EED6F2D8F6DAFADCA7
:10015000FEDE73252034F32510340A8601A07310C7
:10016000153492402241B2414242D2426243F243AC
:10017000025492542255B2554256D2566257F25703
:10018000064896482649B649464AD64A664BF64B33
:10019000065C965C265DB65D465ED65E665FF65F83
:1001A0001301C1077300203010C16374B50011053D
:1001B000E5BF828000000000000000000000000099
:1001C000000000000000000000000000000000002F
:1001D000000000000000000000000000000000001F
:1001E000000000000000000000000000000000000F
:1001F000197106C00AC20EC412C616C81ACA1ECC8D
:1002000022CE26D02AD22ED432D636D83ADA3EDCC6
:1002100042DEC6C0CAC2CEC4D2C6D6C8DACADECC96
:10022000E2CEE6D0EAD2EED4F2D6F6D8FADAFEDCA6
:100230009702020083A2421A23A02200F322103464
:1002400096DEEF006030170102000321E118024141
:10025000F65273901234B72200009382028873A082
:10026000023082403242C2425243E24372448254DC
:100270001255A2553256C2565257E2577258864806
:100280001649A649364AC64A564BE64B764C865C1A
:10029000165DA65D365EC65E565FE65F0961730059
:1002A0002030970202009382E21523A0120023A2BD
:1002B000220023A4320023A6420023A8520023AA2E
:1002C000620023AC720023AE820023A0920223A21C
:1002D000A20223A4B20223A6C20223A8D20223AA06
:1002E000E20223ACF20223AE020323A0120523A2F2
:1002F000220523A4320523A6420523A8520523AADA
:10030000620523AC720523AE820523A0920723A2C7
:10031000A20723A4B20723A6C20723A8D20723AAB1
:10032000E20723ACF207EF40C06A17010200032185
:10033000A10A0241F65273901234B7220000938250
:10034000028873A0023082403242C2425243E243EA
:10035000724482541255A2553256C2565257E25731
:10036000725886481649A649364AC64A564BE64B45
:10037000764C865C165DA65D365EC65E565FE65FB1
:10038000096173002030970202009382A20783A0C4
:10039000020003A1420083A1820003A2C20083A243
:1003A000020103A3420183A3820103A4C20183A427
:1003B000020203A5420283A5820203A6C20283A60B
:1003C000020303A7420383A7820303A8C20383A8EF
:1003D000020403A9420483A9820403AAC20483AAD3
:1003E000020503AB420583AB820503ACC20583ACB7
:1003F000020603AD420683AD820603AEC20683AE9B
:10040000020703AFC20983AF820782807370043092
:10041000197106C00AC20EC412C616C81ACA1ECC6A
:1004200022CE26D02AD22ED432D636D83ADA3EDCA4
:1004300042DEC6C0CAC2CEC4D2C6D6C8DACADECC74
:10044000E2CEE6D0EAD2EED4F2D6F6D8FADAFEDC84
:100450009702020083A242F823A0220086DEEF105A
:10046000F05D17010200032121F70241F65273905B
:100470001234B72200009382028873A002308240B7
:100480003242C2425243E243724482541255A25550
:100490003256C2565257E257725886481649A649F4
:1004A000364AC64A564BE64B764C865C165DA65DD0
:1004B000365EC65E565FE65F0961730020309707BF
:1004C0000200938727F29843FD576305F700737086
:1004D000043001A07370043001A041112AC6B24754
:1004E000739047300100410182804111F327403071
:1004F0003EC673F04330B2473E85410182804111D0
:100500002AC62EC432C2B247F1173EC62247B247AE
:1005100098C3B247938787FA3EC61247B24798C33B
:10052000B247A1173EC68E873E87B24798C3B247EF
:10053000D1173EC6170700001307A7F8B24798C3A4
:10054000B2473E8541018280411106C6EF40E0403E
:10055000EF101032AA8799C3EF10504E0100B2403D
:100560004101828041112AC6B24713878700B247F2
:10057000D8C3B2477D5798C7B24713878700B247A1
:10058000D8C7B24713878700B24798CBB24723A09A
:10059000070001004101828041112AC6B24723A809
:1005A000070001004101828001112AC62EC4B24712
:1005B000DC433ECEA2477247D8C3F2479847A247D2
:1005C00098C7F2479C472247D8C3F247224798C7AB
:1005D000A247324798CBB2479C4313871700B247D4
:1005E00098C301000561828001112AC62EC4A2476A
:1005F0009C433ECC6247FD576316F700B2479C4BC5
:100600003ECE31A8B247A1073ECE21A0F247DC433F
:100610003ECEF247DC439C436247E379F7FEF24764
:10062000D843A247D8C3A247DC43224798C7A24772
:10063000724798C7F2472247D8C3A247324798CBA0
:10064000B2479C4313871700B24798C30100056166
:10065000828001112AC6B2479C4B3ECEB247DC4392
:100660003247184798C7B2479C4732475843D8C3C8
:10067000F247DC4332476316F700B2479847F24728
:10068000D8C3B24723A80700F2479C431387F7FF5C
:10069000F24798C3F2479C433E8505618280797199
:1006A00006D622D42AC62EC4B2473ECEF24781E7F0
:1006B0007370043001A0EF206074F2478043F2476A
:1006C000D85FF247BC43BE853A85EF503006AA8713
:1006D0003307F400F247D8C3F24723AC0702F247CE
:1006E0009843F24798C7F2478043F247DC5F13878D
:1006F000F7FFF247BC43BE853A85EF503003AA8727
:100700003307F400F247D8C7F2477D57F8C3F247E2
:100710007D57B8C7A24799EFF2479C4B8DC7F24768
:10072000C1073E85EF10D05D2A878547631DF7001E
:10073000F13911A8F247C1073E852D35F24793875D
:1007400047023E850535EF20406E85473E85B25015
:10075000225445618280797106D62AC62EC4B2879A
:10076000A303F10002CCB24781E77370043001A00B
:10077000A24799E302CE01A8A2453245EF50007B83
:10078000AA8785073ECEF247938787053E85EF30DF
:10079000C0792ACAD2479DCFA24789E7D24752479C
:1007A00098C331A0D24713878705D24798C3D24751
:1007B0003247D8DFD2472247B8C385455245C535B1
:1007C000D247034771002388E704D24723AA0704CE
:1007D000D2473ECCE24781E77370043001A0E24784
:1007E0003E85B25045618280797106D6AA87A307FB
:1007F000F10013058005EF3040732ACEF247B5C3F0
:10080000F24723A20700F24723A00700F24723A4E0
:100810000700F24723A60700F24723AC0702F2477E
:100820000547D8DFF24723A00704F2477D57F8C3F6
:10083000F2477D57B8C7F2470347F1002388E70422
:10084000F24723AA0704F247C1073E85213BF2473E
:10085000938747023E85393381460146814572457B
:100860003122F2473E85B25045618280797106D6C9
:1008700022D42AC6B2473ECCE24781E773700430E7
:1008800001A0E247C043EF208039AA876313F40236
:10089000E247DC471387F7FFE247D8C7E247DC4768
:1008A00091E78146014681456245C92085473ECE94
:1008B00011A002CEF2473E85B2502254456182809B
:1008C000797106D622D42AC62EC4B2473ECCE2475E
:1008D00081E77370043001A0E247C043EF20203469
:1008E000AA87631BF400E247DC4713871700E2473F
:1008F000D8C785473ECE0DA0814622468145624538
:10090000592E2ACE724785476318F700E247DC4725
:1009100013871700E247D8C7F2473E85B2502254EA
:1009200045618280797106D62AC62EC4B24781E716
:100930007370043001A02247B24763F5E70073707B
:10094000043001A009468145324531352ACEF247AF
:1009500081C7F247224798DFF24781E7737004307E
:1009600001A0F2473E85B25045618280397106DEB2
:100970002AC62EC432C236C002D6B2473ED4A257CF
:1009800081E77370043001A0A24781E7A257BC43FE
:1009900099E3854711A0814781E77370043001A076
:1009A000024789476317F700A257D85F854763144A
:1009B000F700854711A0814781E77370043001A0DB
:1009C000EF204027AA8799E3924799E3854711A032
:1009D000814781E77370043001A0EF202042A257C5
:1009E000985FA257DC5F6366F70002478947631A86
:1009F000F7040246A245225519252AD2A257FC4BDC
:100A000099CB82452255EF0090222A8785476316AD
:100A1000F702ED3A1DA0A257DC5389CFA257938766
:100A200047023E85EF10D02D2A8785476317F700D0
:100A3000F13A21A0925791C3D13AEF20003F854768
:100A400071A8924789E7EF20403E814741A8B257FD
:100A500099E77C083E85EF10504285473ED6EF204F
:100A6000C03CEF102035EF206039A257F843FD5706
:100A70006315F700A25723A20704A257B847FD57F2
:100A80006315F700A25723A40704EF20003A58008B
:100A90007C08BA853E85EF105041AA879DEB225510
:100AA000EF004077AA878DC3A257C1071247BA85C6
:100AB0003E85EF10D00B2255A525EF106031AA8797
:100AC000E39D07F0A13211BF2255992DEF10403060
:100AD00029B72255B125EF10A02F81473E85F2504E
:100AE00021618280797106D62AC62EC432C236C0F0
:100AF000B2473ECCE24781E77370043001A0A247C1
:100B000081E7E247BC4399E3854711A0814781E72C
:100B10007370043001A0024789476317F700E2476A
:100B2000D85F85476314F700854711A0814781E7A7
:100B30007370043001A0553AAA873ECAE247985F15
:100B4000E247DC5F6366F700024789476316F706F2
:100B50000246A24562456521E247B847FD57631446
:100B6000F704E247FC4B99CF82456245EF00300C19
:100B70002A878547631FF702924785CF924705472B
:100B800098C305A8E247DC538DC7E2479387470225
:100B90003E85EF10F016AA8789CF924799CB9247EE
:100BA000054798C339A0E247BC4713871700E247BF
:100BB000B8C785473ECE11A002CED2473E85313A16
:100BC000F2473E85B25045618280797106D62AC6C9
:100BD0002EC4B2473ECCE24781E77370043001A0D7
:100BE000E247BC4381C77370043001A0E2479C43D5
:100BF00081E7E247DC4399E3854711A0814781E71C
:100C00007370043001A0D530AA873ECAE247985FCE
:100C1000E247DC5F6378F706E2479C5F13871700C3
:100C2000E24798DFE247B847FD576314F704E2470D
:100C3000FC4B99CF81456245EF00607F2A8785474D
:100C4000631FF702A24785CFA247054798C305A8AF
:100C5000E247DC538DC7E247938747023E85EF109A
:100C6000300AAA8789CFA24799CBA247054798C3E4
:100C700039A0E247BC4713871700E247B8C785474A
:100C80003ECE11A002CED2473E858138F2473E8546
:100C9000B25045618280397106DE2AC62EC432C246
:100CA00036C002D6B2473ED4A25781E773700430F3
:100CB00001A0A24781E7A257BC4399E3854711A051
:100CC000814781E77370043001A0EF10B076AA87E6
:100CD00099E3924799E3854711A0814781E77370B3
:100CE000043001A0EF208011A2579C5FB5CBA25722
:100CF000DC473ED2A2452255F92E824795EFA257F6
:100D00009C5F1387F7FFA25798DFA2579C4391E798
:100D1000EF2000192A87A257D8C3A2579C4B8DCF2A
:100D2000A257C1073E85EF10A07D2A87854763152E
:100D3000F702EFF0AFED0DA0A2571257D8C7A25798
:100D4000DC5399CBA257938747023E85EF10407B37
:100D5000AA8799C3EFF08FEBEF20200D85475DA8A0
:100D6000924789E7EF20600C81476DA0B25799E761
:100D70007C083E85EF10701085473ED6EF20E00AD4
:100D8000EF104003EF208007A257F843FD5763158B
:100D9000F700A25723A20704A257B847FD576315CF
:100DA000F700A25723A40704EF20200858007C086E
:100DB000BA853E85EF10700FAA87A1EB225531212D
:100DC000AA879DCFA2579C4391EBEF202003A25707
:100DD000DC433E85EF101069EF202005A257938772
:100DE00047021247BA853E85EF10605822550D2EF6
:100DF000EF00107EAA87E39707EEEFF02FE1DDB555
:100E00002255392EEF00D07CF1BD2255112EEF0076
:100E1000307C81473E85F25021618280797106D60F
:100E20002AC62EC432C2B2473ECCE24781E7737075
:100E3000043001A0A24781E7E247BC4399E385471C
:100E400011A0814781E77370043001A0EFF0EFE952
:100E5000AA873ECAE2479C5FA1CBA2456245A52C6A
:100E6000E2479C5F1387F7FFE24798DFE247F843CA
:100E7000FD576312F702E2479C4B85C7E247C10763
:100E80003E85EF10E067AA8789CF924799CB9247BA
:100E9000054798C339A0E247FC4313871700E24790
:100EA000F8C385473ECE11A002CED2473E85EFF073
:100EB000CFE2F2473E85B25045618280797106D615
:100EC0002AC62EC4B2473ECCE24781E77370043095
:100ED00001A0A24781E7E247BC4399E3854711A0FF
:100EE000814781E77370043001A0E247BC4381E78A
:100EF0007370043001A0EFF04FDFAA873ECAE247CB
:100F00009C5F89CFE247DC473EC8A2456245E122AB
:100F1000E2474247D8C785473ECE11A002CED2470E
:100F20003E85EFF08FDBF2473E85B250456182800F
:100F3000797106D62AC6B24781E77370043001A0E2
:100F4000EF10D06BB2479C5F3ECEEF10106EF247B1
:100F50003E85B25045618280797106D62AC6B24775
:100F60003ECEF24781E77370043001A0EF101069A4
:100F7000F247D85FF2479C5FB307F7403ECCEF10D3
:100F8000D06AE2473E85B2504561828001112AC68F
:100F9000B24781E77370043001A0B2479C5F3ECE38
:100FA000F2473E8505618280797106D62AC6B2472E
:100FB0003ECEF24781E77370043001A072450926E6
:100FC0007245EF3080090100B250456182804111C5
:100FD0002AC6B247FC473E854101828041112AC69C
:100FE0002EC4B2472247F8C7010041018280411157
:100FF0002AC6B24783C707053E85410182807971C1
:1010000006D62AC62EC432C202CEB247BC4391EFE6
:10101000B2479C43D5E7B247DC433E85EF103052E0
:101020002ACEB24723A2070061A8924785EFB247B4
:101030009847B247BC433E86A2453A85EF308010C0
:10104000B2479847B247BC433E97B24798C7B247AA
:101050009847B247DC436365F706B2479843B24707
:1010600098C7B9A8B247D847B247BC433E86A24505
:101070003A85EF30200DB247D847B247BC43B3079B
:10108000F0403E97B247D8C7B247D847B2479C43D3
:10109000637BF700B247D843B247BC43B307F04085
:1010A0003E97B247D8C712478947631BF700B2473C
:1010B0009C5F99C7B2479C5F1387F7FFB24798DFE1
:1010C000B2479C5F13871700B24798DFF2473E850F
:1010D000B25045618280011106CE2AC62EC4B247A5
:1010E000BC439DCBB247D847B247BC433E97B247BB
:1010F000D8C7B247D847B247DC436366F700B24768
:101100009843B247D8C7B247D847B247BC433E8698
:10111000BA852245EF3000030100F240056182806C
:10112000011106CE2AC6EF10704D89A0B247FC4BC4
:1011300099CB81453245E52C2A8785476312F70212
:10114000EF10006031A8B247DC5395C7B2479387D0
:1011500047023E85EF10C03AAA8799C3EF10405E60
:10116000B247BC471387F7FFB247B8C7B247BC477F
:10117000E34EF0FA11A00100B2477D57B8C7EF1057
:10118000D04AEF10B0471DA0B2479C4B8DC7B24765
:10119000C1073E85EF10C036AA8799C3EF10405AA9
:1011A000B247FC431387F7FFB247F8C3B247FC438B
:1011B000E34CF0FC11A00100B2477D57F8C3EF10DB
:1011C000D0460100F24005618280797106D62AC6B8
:1011D000EF10D042B2479C5F81E785473ECE11A019
:1011E00002CEEF109044F2473E85B25045618280B6
:1011F00001112AC6B24781E77370043001A0B247DB
:101200009C5F81E785473ECE11A002CEF2473E8526
:1012100005618280797106D62AC6EF10303EB2474A
:10122000985FB247DC5F6315F70085473ECE11A09B
:1012300002CEEF10903FF2473E85B250456182806A
:1012400001112AC6B24781E77370043001A0B2478A
:10125000985FB247DC5F6315F70085473ECE11A06B
:1012600002CEF2473E850561828001112AC62EC456
:1012700002CE81A0178703001307C749F2478E07E4
:10128000BA979C4385E7178703001307A748F247DF
:101290008E07BA97224798C317870300130787471B
:1012A000F2478E07BA973247D8C301A8F24785079D
:1012B0003ECE72479D47E3FFE7FA01000561828059
:1012C00001112AC602CE0DA8178703001307874411
:1012D000F2478E07BA97DC433247631CF700178743
:1012E000030013072743F2478E07BA9723A007008E
:1012F00001A8F24785073ECE72479D47E3F6E7FC1B
:10130000010005618280797106D62AC62EC432C2D8
:10131000B2473ECEEF10902EF247F843FD576315CB
:10132000F700F24723A20704F247B847FD576315B9
:10133000F700F24723A40704EF10302FF2479C5F19
:1013400089EBF247938747021246A2453E85EF108C
:1013500080137245F1330100B2504561828079718A
:1013600006D62AC6014691453245EFF0CFBE2ACEB9
:10137000F2473E85B25045618280797106D62AC611
:101380002EC4EF10B027B247FC4B99C302CE19A868
:10139000B2479C5F99C302CE31A0B2472247F8CB37
:1013A00085473ECEEF107028F2473E85B25045612A
:1013B0008280797106D62AC62EC4B2473ECCE24757
:1013C000FC4B22476304F70002CE39A8E2479C5F3A
:1013D00099C302CE11A8EF107022E24723AA070496
:1013E000EF10B02485473ECEF2473E85B2504561AE
:1013F0008280797106D62AC62EC402CE7C08814628
:101400002246BE8532454138F2473E85B25045619D
:101410008280797106D62AC602CE7C080146BE8536
:101420003245ED3AF2473E85B2504561828079718E
:1014300006D62AC62EC4B247FC4B3ECC02CEE247AB
:1014400081E77370043001A0E247985FE247DC5FF8
:101450006365F7007370043001A0E247985FE247CC
:10146000DC5F6371F7047C002246BE856245413E25
:101470002ACEE247B847FD576310F702E247DC5334
:1014800095C3E247938747023E85EF106007AA871E
:1014900091CB85473ECE39A0E247BC471387170062
:1014A000E247B8C7F2473E85B25045618280397144
:1014B00006DE2ACE2ECC36C83AC63EC442C246C04C
:1014C000B287231BF100F24781E77370043001A05B
:1014D0003247A54763F5E7007370043001A08357D6
:1014E000610192453E85EF1080512AD4A257638F47
:1014F0000712A257985B83566101B7070040FD179A
:10150000B6978A07BA973ED29257F19B3ED292572E
:101510008D8B81C77370043001A0835761013E87B2
:1015200082463246E2452255EF10E0274246F24518
:101530001255EFE0DFFC2A87A25798C3A24781C764
:10154000A247225798C3EF10700B97F701009387BB
:10155000A7069C431387170097F701009387C705D9
:1015600098C397F70100938727E79C4395E397F784
:101570000100938767E6225798C397F70100938786
:10158000A70398438547631AF702EF10C02C35A0D4
:1015900097F70100938707039C4385E397F70100C2
:1015A000938787E39C43DC5732476368F70097F7DC
:1015B0000100938767E2225798C397F7010093874A
:1015C00067019C431387170097F7010093878700F3
:1015D00098C397F701009387E7FF9843A257B8C7CE
:1015E000A257D85797F70100938787FD9C4363F96B
:1015F000E700A257D85797F70100938767FC98C375
:10160000A257D857BA878A07BA978A0717F70100EF
:10161000130707E73E97A2579107BE853A85EFE08B
:10162000BFF885473ED6EF10500019A0FD573ED6B3
:10163000325785476313F70297F70100938787F8BE
:101640009C4381CF97F70100938707D99C43DC57D0
:10165000324763F4E700EFE07FDBB2573E85F2509C
:1016600021618280797106D62AC6EF102079B247AF
:1016700099E797F70100938727D69C4311A0B247BB
:101680003ECEF24791073E85EFE0BFFCF2479C5704
:1016900091C7F247E1073E85EFE0BFFBF2479107B4
:1016A000BE8517F50100130565EEEFE0FFEF97F734
:1016B00001009387E7EE9C431387170097F701001B
:1016C000938707EE98C397F701009387A7F09C4391
:1016D0001387170097F701009387C7EF98C3EF10A0
:1016E000C07497F701009387E7ED9C439DCB97F774
:1016F0000100938767CE9C437247631EF70097F7FC
:1017000001009387A7ED9C4381C77370043001A04B
:10171000EFE0DFCF39A0EF10606EEF10A04BEF10BD
:10172000C0700100B25045618280797106D62AC628
:101730002EC402CEB24781E77370043001A0A247E5
:1017400081E77370043001A097F70100938707E9E0
:101750009C4381C77370043001A0A92D97F7010045
:101760009387C7E59C433ECCB2479C432247BA9738
:101770003ECAB2479C436247637EF700B2479C4330
:1017800052476374F7025247E24763F0E702854726
:101790003ECE21A8B2479C4352476366F7005247AA
:1017A000E24763F4E70085473ECEB247524798C30D
:1017B000F24789CF97F70100938707C29C439107AF
:1017C0003E85EFE01FE95245EF10001B11252AC8A6
:1017D000C24799E3EFE09FC30100B25045618280A8
:1017E000797106D62AC602CEB247A9C397F701007F
:1017F0009387C7DE9C4381C77370043001A05D2BC3
:1018000097F70100938787DB9C433247BA973ECC1A
:1018100097F70100938747BC9C4391073E85EFE013
:101820005FE36245EF10401565232ACEF24799E346
:10183000EFE0DFBD0100B25045618280797106D6CC
:101840002AC6B2473ECCE24781E77370043001A05C
:1018500097F70100938747B89C4362476314F700EA
:1018600002CEBDA0EF108059E247DC4B3ECAEF101C
:10187000C05B97F701009387A7CF9C435247630A49
:10188000F70097F701009387E7CE9C435247631513
:10189000F70089473ECE2DA8524797F7010093875E
:1018A00067D0631BF700E2479C5781E78D473ECE28
:1018B00005A089473ECE29A8524797F70100938794
:1018C000E7CC6315F70091473ECE19A085473ECE81
:1018D000F2473E85B25045618280797106D62AC6AC
:1018E000EF10C051B24799E797F701009387C7AE51
:1018F0009C4311A0B2473ECEF247DC573ECCEF10DE
:10190000C052E2473E85B25045618280797106D669
:101910002AC6EFE09FBDAA873ECEB24799E797F768
:101920000100938767AB9C4311A0B2473ECCE247CE
:10193000DC573ECAF2473E85EFE03FBAD2473E85CC
:10194000B25045618280797106D62AC62EC402CE75
:101950002247A54763F5E7007370043001A02247D2
:10196000A54763F4E700A5473EC4EF102049B247FE
:1019700099E797F70100938727A69C4311A0B247E8
:101980003ECCE247BC4B3ECA5247A247630AF70E21
:101990002247D24763F6E70297F701009387C7A370
:1019A0009C4362476308F70297F701009387C7A239
:1019B0009C43DC572247636FF70085473ECE19A84A
:1019C00097F70100938747A19C4362476314F70090
:1019D00085473ECEE247DC573EC8E247B84BE24778
:1019E000DC576315F700E2472247D8D7E247224782
:1019F000B8CBE2479C4F63C707002947A2471D8F1A
:101A0000E24798CFE247D44B4247BA878A07BA9752
:101A10008A0717F701001307A7A6BA976394F60081
:101A2000854711A08147B9C7E24791073E85EFE09E
:101A30005FC2E247D85797F70100938767B89C4386
:101A400063F9E700E247D85797F70100938747B754
:101A500098C3E247D857BA878A07BA978A0717F711
:101A600001001307E7A13E97E2479107BE853A853B
:101A7000EFE09FB3724785476314F700EFE01F99CB
:101A8000EF10A03A0100B25045618280797106D60C
:101A90002AC6EF10A036B24799E797F7010093875F
:101AA000A7939C4311A0B2473ECEF24791073E85D3
:101AB000EFE03FBAF2479C5791C7F247E1073E85F6
:101AC000EFE03FB9F2479107BE8517F50100130516
:101AD00065ADEFE07FADEF10403597F701009387DC
:101AE000A78F9C4372476319F70497F70100938708
:101AF00067AD9C4389CF97F70100938727AE9C433E
:101B000081C77370043001A0EFE05F9091A097F758
:101B10000100938727A9984397F701009387C7A9E6
:101B20009C436319F70097F701009387E78A23A086
:101B3000070039A8212729A897F70100938787A8CC
:101B40009C4399C7EF10802BEF10C008EF10E02DD9
:101B50000100B2504561828001112AC602CEB2470F
:101B60003ECCB24781E77370043001A0E247D84B06
:101B700097F70100938707A36314F700854711A027
:101B8000814795C3E247985797F701009387C79E0F
:101B9000630BF700E2479C5799E3854711A0814703
:101BA00099C385473ECEF2473E85056182807971B3
:101BB00006D62AC6B2473ECEB24781E773700430DC
:101BC00001A0F247C9C797F701009387E7809C43BC
:101BD0007247630EF706EF1060227245B53F2A8701
:101BE00085476314F706F24791073E85EFE07FA62D
:101BF000F247D85797F701009387879C9C4363F976
:101C0000E700F247D85797F701009387679B98C37F
:101C1000F247D857BA878A07BA978A0717F7010099
:101C2000130707863E97F2479107BE853A85EFE096
:101C3000BF97F247D85797E701009387E7799C430E
:101C4000DC576364F700EFE06FFCEF10001E01004B
:101C5000B25045618280797106D62AC602CEB2475B
:101C60003ECCB24781E77370043001A0EFE0FF87FC
:101C7000AA873ECA6245CD352A8785476314F7088F
:101C800097F70100938787959C43A5E7E247D857CC
:101C900097E70100938747749C43DC576364F70020
:101CA00085473ECEE24791073E85EFE09F9AE247A7
:101CB000D85797F701009387A7909C4363F9E700F3
:101CC000E247D85797F701009387878F98C3E24779
:101CD000D857BA878A07BA978A0717E70100130708
:101CE000277A3E97E2479107BE853A85EFE0DF8B82
:101CF00011A8E247E107BE8517F501001305C58766
:101D0000EFE09F8AD2473E85EFE02FFDF2473E8508
:101D1000B25045618280011106CE81480148814759
:101D2000014781461306004097E501009385852D04
:101D300017150000130585A5EFF06FF72AC6324787
:101D400085476315F700EF10C06D2AC632478547F7
:101D50006319F7027370043097F701009387C78700
:101D60007D5798C397F701009387C785054798C3A8
:101D700097F701009387878423A00700EFE06FD2D5
:101D800031A0B24781E77370043001A00100F24036
:101D900005618280411106C67370043097F7010017
:101DA0009387478223A00700EFE0EFDD0100B240F8
:101DB0004101828097F70100938747829C431387F4
:101DC000170097F701009387678198C3010082800D
:101DD000011106CE02C697F70100938727809C4326
:101DE00081E77370043001A0EF10400197E7010014
:101DF0009387C77E9C431387F7FF97E7010093877C
:101E0000E77D98C397E701009387477D9C436390E4
:101E1000071097E701009387277A9C436389070E91
:101E200059A097E7010093872775DC47DC473EC43C
:101E3000A247E1073E85EFE0DF81A24791073E859B
:101E4000EFE03F81A247D85797E701009387477794
:101E50009C4363F9E700A247D85797E701009387AF
:101E6000277698C3A247D857BA878A07BA978A07AE
:101E700017E701001307C7603E97A2479107BE8589
:101E80003A85EFE06FF2A247D85797E701009387B2
:101E9000A7549C43DC576368F70097E701009387DA
:101EA000E772054798C397E701009387E76C9C4367
:101EB000ADFB97E70100938727719C438DCF35A039
:101EC000452AAA8799C797E7010093872770054796
:101ED00098C397E701009387276F9C431387F7FF09
:101EE00097E701009387476E98C397E701009387B0
:101EF000A76D9C43F1F797E701009387276D9843FF
:101F000085476316F70085473EC6EFE02FD0EF0008
:101F1000D071B2473E85F24005618280011106CE44
:101F2000EF00D06D97E70100938747699C433EC659
:101F3000EF00B06FB2473E85F2400561828001112B
:101F400006CEEFE08FDAAA873EC697E701009387B7
:101F5000E7669C433EC4B2473E85EFE00FD8A247F8
:101F60003E85F2400561828097E701009387C76450
:101F70009C433E858280797106D62AC62EC432C221
:101F800002CEA9473ECC3D3597E701009387C76253
:101F90009C4322476368F70CE247FD173ECCF247AB
:101FA00096073247B306F7006247BA878A07BA979F
:101FB0008A0717E701001307A74CBA970546BE85A5
:101FC0003685EF00902A2A87F247BA973ECEE2473D
:101FD000E1F7F247960732473E9797E7010093876C
:101FE00027599C430946BE853A85EF0010282A8769
:101FF000F247BA973ECEF247960732473E9797E7A9
:102000000100938727579C430946BE853A85EF0018
:10201000D0252A87F247BA973ECEF2479607324735
:10202000BA97114697E50100938545563E85EF0026
:10203000D0232A87F247BA973ECEF2479607324717
:10204000BA970D4697E501009385C5553E85EF008B
:10205000D0212A87F247BA973ECE924781C792474E
:1020600023A00700B533F2473E85B2504561828018
:10207000797106D602CE97E70100938727569C43D5
:102080006395071897E70100938747539C4313878D
:10209000170097E701009387675298C397E70100FD
:1020A0009387C7519C433ECCE247B9EF97E70100C5
:1020B0009387074C9C439C4381C77370043001A0F5
:1020C00097E701009387C74A9C433ECA97E7010000
:1020D0009387474A984397E701009387674998C3D6
:1020E00097E7010093870749524798C397E7010094
:1020F0009387074E9C431387170097E70100938748
:10210000274D98C3EF00102D97E701009387C74C28
:102110009C4362476365F70C97E701009387474547
:102120009C439C4399E3854711A0814781CB97E766
:1021300001009387674A7D5798C355A097E7010030
:10214000938707439C43DC47DC473EC8C247DC43D8
:102150003EC66247B2476379F70097E7010093876D
:10216000A747324798C3A5A8C24791073E85EFE02D
:102170004FCEC2479C5791C7C247E1073E85EFE06B
:102180004FCDC247D85797E70100938767439C43D9
:1021900063F9E700C247D85797E7010093874742A2
:1021A00098C3C247D857BA878A07BA978A0717E7EA
:1021B00001001307E72C3E97C2479107BE853A8579
:1021C000EFE08FBEC247D85797E701009387C7203B
:1021D0009C43DC57E362F7F485473ECE35BF97E773
:1021E00001009387671F9C43D85797E601009386A9
:1021F0002629BA878A07BA978A07B69798438547E8
:1022000063F1E70285473ECE29A897E7010093874F
:10221000A73B9C431387170097E701009387C73AB2
:1022200098C397E701009387673A9C4399C3854712
:102230003ECEF2473E85B25045618280011106CE06
:1022400097E70100938787399C4381CB97E701008B
:102250009387C737054798C339A297E7010093874B
:10226000E73623A0070097E701009387E7169C4312
:102270009C5B3EC6B7A7A5A59387575A3EC4B247F5
:102280009C4322476314F702B24791079C432247BD
:10229000631EF700B247A1079C4322476318F7006B
:1022A000B247B1079C4322476308F70497E7010050
:1022B00093878712984397E701009387E7119C4320
:1022C00093874703BE853A85EF20F00F35A097E747
:1022D00001009387E72E9C4381E77370043001A0CF
:1022E00097E701009387C72D9C431387F7FF97E774
:1022F00001009387E72C98C397E701009387472C49
:10230000984397E601009386A617BA878A07BA977B
:102310008A07B6979C43C5DF97E701009387472A52
:102320009843BA878A07BA978A0717E70100130705
:102330002715BA973EC29247DC43D8439247D8C389
:102340009247D8439247A1076317F7009247DC43AF
:10235000D8439247D8C39247DC43D84797E7010058
:102360009387870798C30100F240056182807971E5
:1023700006D62AC62EC4B24781E77370043001A086
:1023800097E70100938747059C43E107BE853245E7
:10239000EFE08FA597E70100938707049C4391071F
:1023A0003E85EFE00FAB2247FD576310F70297E73A
:1023B0000100938767029C439107BE8517E50100E2
:1023C0001305451EEFE04F9E19A897E7010093877C
:1023D000E71E9C432247BA973ECE7245712B0100FF
:1023E000B25045618280797106D62AC62EC432C2A7
:1023F000B24781E77370043001A097E7010093872B
:10240000E71D9C4381E77370043001A097E701004A
:10241000938787FC9C43A24637070080558F98CF4F
:1024200097E70100938747FB9C43E107BE85324550
:10243000EFE08F9797E70100938707FA9C43910796
:102440003E85EFE00FA11247FD576310F70297E7B3
:102450000100938767F89C439107BE8517E501004B
:1024600013054514EFE04F9419A897E701009387EF
:10247000E7149C431247BA973ECE7245F5290100F6
:10248000B25045618280797106D62AC62EC432C206
:10249000B24781E77370043001A097E7010093878A
:1024A000A7F39C43E107BE853245EFE0EF8F97E746
:1024B0000100938767F29C4391073E85EFE06F9997
:1024C000124785476310F70297E701009387C7F02B
:1024D0009C439107BE8517E501001305A50CEFE0AD
:1024E000AF8C19A897E701009387470D9C432247BB
:1024F000BA973ECE724549210100B25045618280B3
:10250000797106D62AC6B247DC47DC473ECCE247A3
:1025100081E77370043001A0E247E1073E85EFE0F8
:102520004F9397E701009387670B9C43A1EBE2472A
:1025300091073E85EFE0EF91E247D85797E701001A
:10254000938707089C4363F9E700E247D85797E76A
:1025500001009387E70698C3E247D857BA878A07EE
:10256000BA978A0717E70100130787F13E97E247FA
:102570009107BE853A85EFE02F8311A8E247E10776
:10258000BE8517E50100130525FFEFE0EF81E24767
:10259000D85797E70100938727E49C43DC5763FBF8
:1025A000E70085473ECE97E701009387270205475E
:1025B00098C311A002CEF2473E85B2504561828099
:1025C000797106D62AC62EC497E7010093870701C2
:1025D0009C4381E77370043001A02247B707008055
:1025E0005D8FB24798C3B247DC473ECCE24781E7F4
:1025F0007370043001A03245EFE0AF85E2479107E8
:102600003E85EFE00F85E247D85797E701009387B3
:1026100027FB9C4363F9E700E247D85797E701009F
:10262000938707FA98C3E247D857BA878A07BA97B9
:102630008A0717E701001307A7E43E97E2479107CF
:10264000BE853A85EFD05FF6E247D85797E701009D
:10265000938787D89C43DC5763FBE70085473ECED2
:1026600097E70100938787F6054798C311A002CE2C
:10267000F2473E85B2504561828041112AC6B24779
:1026800081E77370043001A097E70100938747F456
:102690009843B24798C397E70100938727F298437E
:1026A000B247D8C3010041018280797106D62AC69B
:1026B0002EC4B24781E77370043001A0A24781E7BE
:1026C0007370043001A01D2F97E70100938707EF77
:1026D0009C433ECCA2479843FD576314F70002CEBB
:1026E00091A8B247984397E70100938767EE9C4310
:1026F000630AF700B247DC4362476365F70085472A
:102700003ECE0DA8B247DC4362471D8FA2479C43D3
:102710006370F702A2479843B247D443E247B387B6
:10272000F6403E97A24798C33245813F02CE19A09A
:1027300085473ECEDD2DF2473E85B2504561828011
:1027400097E70100938787E8054798C301008280D7
:1027500001112AC6B24799C7B2473ECCE247FC47AF
:102760003ECE11A002CEF2473E8505618280011166
:102770002AC62EC4B24791C7B2473ECEF24722477F
:10278000F8C7010005618280011106CE2AC68522A4
:1027900097E701009387C7CE98438547E3F9E7FEA3
:1027A000EFD0DFC6EDB7397106DE2ACE2ECC32CAA5
:1027B00036C8BA872317F10002D625A06247B25760
:1027C000BA9703C70700F246B257B697238AE702C3
:1027D0006247B257BA9783C7070089CBB2578507BC
:1027E0003ED63257BD47E3FBE7FC11A00100F2479C
:1027F000A38107045247A54763F4E700A5473ECAF3
:10280000F2475247D8D7F2475247B8CBF24723AAEC
:102810000704F24791073E85EFD01FD8F247E10742
:102820003E85EFD07FD7F247724798CB2947D247F2
:102830001D8FF24798CFF2477247D8D3F24723A2B1
:102840000704F24723AC0704F24723AE0704010054
:10285000F25021618280011106CE02C60DA03247DE
:10286000BA878A07BA978A0717E70100130747C193
:10287000BA973E85EFD01FCFB24785073EC6324795
:10288000A547E3FEE7FC17E501001305E5CBEFD014
:102890007FCD17E50100130565CCEFD0BFCC17E560
:1028A0000100130565CDEFD0FFCB17E5010013053F
:1028B000E5CDEFD03FCB17E501001305A5CEEFD056
:1028C0007FCA97E701009387A7CA17E7010013079C
:1028D000A7C798C397E701009387C7C917E7010007
:1028E0001307C7C798C30100F24005618280011138
:1028F00006CE8DA8EFF00FCC97E70100938707C9AC
:102900009C4393B7170093F7F70F3EC6EFF04FCCF9
:10291000B247A9EBE52197E70100938727C7DC477A
:10292000DC473EC4A24791073E85EFD09FD297E790
:102930000100938767C89C431387F7FF97E701005F
:10294000938787C798C397E70100938767C59C4320
:102950001387F7FF97E70100938787C498C3F12196
:102960002245912C97E70100938787C39C43D9F3B5
:102970000100F24005618280011106CE2AC697E768
:102980000100938767A59C433247D8C397E70100AE
:102990009387C7C29C4332476372F70297E70100EF
:1029A000938747BD984397E701009387E7A29C432D
:1029B0009107BE853A85EFD03FC335A897E7010060
:1029C000938707BB984397E701009387E7A09C4351
:1029D0009107BE853A85EFD03FC197E70100938705
:1029E000A7BF9C4332476378F70097E701009387BE
:1029F000A7BE324798C30100F24005618280797119
:102A000006D6AA872EC42317F100A24789EB835765
:102A1000E1008A073E85EF104051AA8711A0A24726
:102A20003ECCE24785C313050006EF1000502ACEC6
:102A3000F24789C7F247624798DB31A06245EF1041
:102A4000C06111A002CEF24781CFF247985B835755
:102A5000E1008A073E869305500A3A85EF104075DB
:102A6000F2473E85B25045618280397106DE22DC34
:102A70002AC62EC432C202D6A2479C43638D070EDB
:102A8000A2473ED4A257DC43D843A257D8C3A2578B
:102A9000D843A257A1076317F700A257DC43D843D6
:102AA000A257D8C3A257DC43DC473ED2A2473ED050
:102AB0008257DC43D8438257D8C38257D8438257C2
:102AC000A1076317F7008257DC43D8438257D8C366
:102AD0008257DC43DC473ECEB25796073247BA975F
:102AE000724798C3B25796073247BA97724713078F
:102AF0004703D8C3B25796073247BA977247384749
:102B000098C7B25796073247BA971247D8C7B257F5
:102B100096073247BA977247585798CB12478D4756
:102B2000631BF700F2479C5799C7B2579607324785
:102B3000BA970947D8C7B25796073247BA9772472C
:102B4000384BD8CBB25796073247BA9723AC070019
:102B5000F247945BB257960732473304F700368545
:102B60000D20AA87231EF400B25785073ED6724770
:102B70009257E31DF7F2B2573E85F250625421613D
:102B8000828001112AC602CE39A0B24785073EC60F
:102B9000F24785073ECEB24703C707009307500AA6
:102BA000E305F7FEF24789833ECEF247C207C183B1
:102BB0003E8505618280011106CE2AC6B2479C5B24
:102BC0003E85EF1080493245EF1020490100F24068
:102BD00005618280411197E70100938767999C43C3
:102BE0009C4399E3854711A0814781CB97E701007A
:102BF0009387879E7D5798C305A097E70100938729
:102C000027979C43DC47DC473EC6B247D84397E74B
:102C100001009387679C98C30100410182804111A4
:102C200097D701009387477B9C433EC6B2473E85BA
:102C300041018280411197E701009387A7989C4347
:102C400081E785473EC619A897E701009387079952
:102C50009C4381E789473EC611A002C6B2473E8524
:102C600041018280797106D62AC6B2473ECEB2476C
:102C7000F9C3F247D85797D701009387E7759C436C
:102C8000DC57637AF70AF2479C4F63CC070097D76B
:102C90000100938767749C43DC5729471D8FF247D7
:102CA00098CFF247D44BF247D857BA878A07BA97DA
:102CB0008A0717D701001307A77CBA976394F60019
:102CC000854711A08147A5C3F24791073E85EFD004
:102CD0005F9897D70100938727709C43D857F24796
:102CE000D8D7F247D85797E701009387678D9C4361
:102CF00063F9E700F247D85797E701009387478CBD
:102D000098C3F247D857BA878A07BA978A0717D75E
:102D100001001307E7763E97F2479107BE853A8593
:102D2000EFD09F8809A897D701009387E76A9C4353
:102D3000D857F247D8D70100B250456182807971E7
:102D400006D62AC6B2473ECC02CEB247DDC397D7DD
:102D50000100938767689C4362476305F7007370BF
:102D6000043001A0E247FC4B81E77370043001A0FE
:102D7000E247FC4B1387F7FFE247F8CBE247D8570F
:102D8000E247BC4B6307F706E247FC4BBDE3E24773
:102D900091073E85EFD0FF8BE247B84BE247D8D78B
:102DA000E247DC5729471D8FE24798CFE247D857C3
:102DB00097E701009387C7809C4363F9E700E247E8
:102DC000D85797D701009387A77F98C3E247D85772
:102DD000BA878A07BA978A0717D701001307476A85
:102DE0003E97E2479107BE853A85EFD0EFFB8547D6
:102DF0003ECEF2473E85B25045618280737004300A
:102E000097D701009387077C9C4391CF97D7010008
:102E10009387875C9C43F8430507F8C397D7010065
:102E20009387875B9C430100828097D7010093873B
:102E300067799C438DCB97D701009387E7599C43D3
:102E4000FC4395C397D70100938707599C43F843E8
:102E50007D17F8C397D70100938707589C43FC431D
:102E600099E37360043001008280411197D701001B
:102E7000938787569C439C4F3EC697D70100938704
:102E8000A7559C43D85797D701009387E7549C4395
:102E9000A9463387E64098CFB2473E8541018280FC
:102EA00097D70100938747539C4389CB97D701005D
:102EB000938787529C43F84B0507F8CB97D70100BF
:102EC000938787519C433E858280797106D62AC6B6
:102ED0002EC42D3797D70100938707509C43BC4FD2
:102EE000ADE397D701009387274F9C430547F8CF61
:102EF000A247A1CB97D701009387074E9C43910728
:102F00003E85EFD00FF52247FD576310F70297D7A4
:102F100001009387674C9C439107BE8517D501003C
:102F200013054568EFD04FE819A897D7010093879C
:102F3000E7689C432247BA973ECE7245353CEFD0B6
:102F4000EFCCE535653D97D701009387E7489C4373
:102F5000BC4F3ECCE2479DC3B24789CB97D7010017
:102F6000938787479C4323AC070409A897D70100A0
:102F7000938787469C43B84F7D17B8CF97D70100FA
:102F8000938787459C4323AE07044535E2473E853A
:102F9000B25045618280797106D62AC62EC432C2EB
:102FA00036C0A93D97D70100938707439C43F84F4C
:102FB0008947630DF70697D701009387E7419C4344
:102FC000B44F32471347F7FF758FB8CF97D701003B
:102FD000938787409C430547F8CF8247A1CB97D77B
:102FE00001009387673F9C4391073E85EFD06FE6D2
:102FF0000247FD576310F70297D701009387C73D3B
:103000009C439107BE8517D501001305A559EFD044
:10301000AFD919A897D701009387475A9C43024715
:10302000BA973ECC6245893AEFD04FBEFD3BF933AB
:10303000924789CB97D701009387073A9C43B84FB3
:10304000924798C397D70100938707399C43F84F5D
:1030500085476314F70002CE31A897D70100938704
:10306000A7379C43B44F22471347F7FF758FB8CF5C
:1030700085473ECE97D70100938707369C4323AE02
:1030800007046533F2473E85B2504561828079710D
:1030900006D62AC62EC432C236C085473ECEB247B7
:1030A00081E77370043001A0B2473ECC813B824778
:1030B00089C7E247B84F824798C3E247FC4F3ECAF0
:1030C000E2470947F8CF1247914763EEE70492477A
:1030D0001397270097D70100938747F3BA97984330
:1030E00097D70100938787F2BA978287E247B84F54
:1030F000A2475D8FE247B8CF3DA0E247BC4F1387A0
:103100001700E247B8CF05A0E2472247B8CF21A871
:10311000524789476306F700E2472247B8CF21A00C
:1031200002CE11A0010052478547631AF706E24715
:1031300091073E85EFD0EFD1E247D85797D70100EE
:10314000938707489C4363F9E700E247D85797D72E
:1031500001009387E74698C3E247D857BA878A07A2
:10316000BA978A0717D70100130787313E97E247BE
:103170009107BE853A85EFD02FC3E2479C5781C7A0
:103180007370043001A0E247D85797D701009387A6
:10319000A7249C43DC5763F4E700EFD02FA77131DD
:1031A000F2473E85B25045618280397106DE2ACEF3
:1031B0002ECC32CA36C83AC685473ED6F24781E79A
:1031C0007370043001A0F2473ED4EFD00FB2AA874B
:1031D0003ED2C24789C7A257B84FC24798C3A25729
:1031E000FC4F3ED0A2570947F8CF5247914763EEB4
:1031F000E704D2471397270097D70100938747E248
:10320000BA97984397D70100938787E1BA97828747
:10321000A257B84FE2475D8FA257B8CF3DA0A25743
:10322000BC4F13871700A257B8CF05A0A25762471B
:10323000B8CF21A8025789476306F700A257624713
:10324000B8CF21A002D611A0010002578547631D07
:10325000F708A2579C5781C77370043001A097D715
:1032600001009387A7379C43A1EBA25791073E85A6
:10327000EFD02FBEA257D85797D701009387473476
:103280009C4363F9E700A257D85797D7010093876B
:10329000273398C3A257D857BA878A07BA978A079D
:1032A00017D701001307C71D3E97A2579107BE8588
:1032B0003A85EFD06FAF11A8A257E107BE8517D5A9
:1032C00001001305652BEFD02FAEA257D85797D723
:1032D0000100938767109C43DC5763F7E700B24710
:1032E00081C7B247054798C392573E85EFD0EF9EFE
:1032F000B2573E85F25021618280797106D62AC686
:103300002EC4B24781E77370043001A0B2473ECEAD
:10331000EFD0AF9DAA873ECCF247FC4F3ECAF247A2
:103320000947F8CFF247BC4F13871700F247B8CFD1
:1033300052478547631DF708F2479C5781C7737052
:10334000043001A097D70100938747299C43A1EB44
:10335000F24791073E85EFD0CFAFF247D85797D7C6
:1033600001009387E7259C4363F9E700F247D857AC
:1033700097D701009387C72498C3F247D857BA87D5
:103380008A07BA978A0717D701001307670F3E9776
:10339000F2479107BE853A85EFD00FA111A8F247F9
:1033A000E107BE8517D501001305051DEFD0CF9F9E
:1033B000F247D85797D70100938707029C43DC5701
:1033C00063F7E700A24781C7A247054798C3E247D2
:1033D0003E85EFD08F900100B250456182807971B7
:1033E00006D62AC6B2473ECCE24799E797D70100F6
:1033F000938787FE9C4311A0E2473ECC0134E2470D
:10340000F84F89476318F700E24723AE0704854762
:103410003ECE11A002CE113CF2473E85B25045612E
:103420008280011106CE02C61D2B97D7010093871B
:10343000271E9C439DC38148014881470947814617
:103440001306004097D501009385C5BE17050000FF
:103450001305051BEFE0AF852AC6B24781E77370FD
:10346000043001A0B2473E85F24005618280397187
:1034700006DE2ACE2ECC32CA36C83AC6E24799E3D7
:1034800002D62DA81305C002EF00302A2AD6B25763
:1034900095C7F121B257724798C3B257624798CF88
:1034A000B2575247D8CFB257424798D3B257324754
:1034B000D8D3B25791073E85EFD00F8EE24781E710
:1034C0007370043001A0B2573E85F25021618280B2
:1034D000397106DE2ACE2ECC32CA36C83AC602D69A
:1034E000F24781E77370043001A097D701009387FA
:1034F00027129C43B5CBE2473ED0D2473ED2F2479B
:103500003ED46247954763C4E704EFF0AFF22A87E1
:1035100089476310F70297D701009387670F9C4391
:10352000181081463246BA853E85EFD02FC42AD680
:1035300025A897D701009387A70D9C4318108146B3
:103540000146BA853E85EFD06FC22AD631A897D7FB
:1035500001009387E70B9C43181081464246BA85C9
:103560003E85EFD02FD82AD6B2573E85F250216142
:10357000828001112AC6B2473ECEB24781E77370FE
:10358000043001A0F2479C433E8505618280797139
:1035900006D62AC62EC497D701009387E7069C4318
:1035A000DC47DC473ECEF24791073E85EFD06F8A7D
:1035B000F247D84F8547631BF702F247984FB2474F
:1035C000BA97B2462246BE857245B9222A878547F8
:1035D000631EF70001478146324681457245CD3D65
:1035E0002ACCE24781E77370043001A0F247DC5334
:1035F000724582970100B25045618280797106D68A
:103600002AC63C083E8541282ACEE247BE8572453F
:1036100019206922FDB7797106D62AC62EC4EFE0BB
:103620006FF93C083E8545282ACEE247B9EFA2470C
:1036300099EB3247F24763E8E700EFE06FF9F245B4
:103640003245B137A9A0A24781CF97D70100938710
:10365000E7FB9C439C4393B7170093F7F70F3EC4D7
:1036600097D701009387C7FA94433247F247B307CD
:10367000F7402246BE853685EFD0FFC8EFE04FF514
:10368000AA8791E7EFC09FD819A0EFE06FF401007F
:10369000B2504561828001112AC697D701009387F5
:1036A000A7F69C439C4393B7170093F7F70F3E8709
:1036B000B24798C3B2479C4391EB97D701009387D9
:1036C000A7F49C43DC479C433ECE11A002CEF247B8
:1036D0003E8505618280797106D62AC6EFE01F8497
:1036E0002ACE97D701009387E7F29C43724763770E
:1036F000F700692AB247054798C321A0B24723A023
:10370000070097D701009387E7F0724798C3F24705
:103710003E85B25045618280797106D62AC62EC494
:1037200032C236C002CEB2472247D8C3B247324770
:1037300098CB2247924763E8E702124782471D8FE2
:10374000B2479C4F6365F70085473ECE99A097D757
:1037500001009387A7EB9843B2479107BE853A854E
:10376000EFC09FE83DA0124782476379F7002247E8
:1037700082476365F70085473ECE21A897D70100B1
:10378000938787E89843B2479107BE853A85EFC093
:10379000BFE5F2473E85B25045618280797106D619
:1037A000D9A0A24763C0070CC2473ECEF247DC4B0C
:1037B00091C7F24791073E85EFC0BFE95C003E85A7
:1037C000193F2ACCA2472547636FF70813972700B4
:1037D00097D7010093878786BA97984397D70100B8
:1037E0009387C785BA9782873247F2479C4FBA972B
:1037F0003247BA866246BE857245393F2A87854779
:103800006313F706F247DC5372458297F247D84FAD
:103810008547631AF7043247F2479C4FBA9701472E
:1038200081463E868145724565312ACAD24785EF79
:103830007370043001A03247F24798CFF2479C4F93
:1038400081E77370043001A0F247984FE247BA97BE
:10385000E2466246BE857245C13531A07245EF0031
:10386000C07F11A0010097D70100938767DA9C43BE
:10387000380081460146BA853E85EFD0CFC1AA8780
:10388000E39107F20100B25045618280797106D65A
:1038900071A097D70100938727D79C43DC479C43AF
:1038A0003ECC97D70100938727D69C43DC47DC4763
:1038B0003ECAD24791073E85EFC0BFD9D247DC53FD
:1038C00052458297D247D84F85476319F704D247AC
:1038D0009C4F6247BA973EC84247E24763F4E7020B
:1038E000D2474247D8C3D247524798CB97D7010017
:1038F000938787D19843D2479107BE853A85EFC019
:10390000BFCE29A801478146624681455245C93646
:103910002AC6B24781E77370043001A097D701002F
:10392000938787CE9C439C43ADF797D7010093873D
:10393000A7CD9C433ECE97D70100938727CD9843D0
:1039400097D70100938747CC98C397D701009387F7
:10395000E7CB724798C30100B250456182804111A4
:1039600006C6EFF0AFC997D70100938767CA9C439B
:10397000C9E717D501001305A5C6EFC0BFBE17D50F
:103980000100130525C7EFC0FFBD97D7010093873E
:10399000A7C717D701001307A7C498C397D701007B
:1039A0009387C7C617D701001307C7C498C301463A
:1039B000B1451145EFC03FDA2A8797D701009387B9
:1039C00027C598C397D70100938787C49C4381E795
:1039D0007370043001A097D70100938767C39C439D
:1039E00089CF97D701009387A7C29C4397C5010051
:1039F000938545673E85EFD05F87EFF00FC30100E9
:103A0000B24041018280797106D62AC6B2473ECEC5
:103A1000B24781E77370043001A0EFF02FBEF24788
:103A2000DC4BB337F00093F7F70F3ECCEFF0EFBF6E
:103A3000E2473E85B25045618280797106D62AC63A
:103A4000B2473ECEB24781E77370043001A0EFF079
:103A5000EFBAF2479C533ECCEFF02FBDE2473E85D4
:103A6000B25045618280797106D62AC62EC4B2470B
:103A70003ECEB24781E77370043001A0EFF00FB87B
:103A8000F247224798D3EFF04FBA0100B250456198
:103A90008280011106CE714549292AC6B24789CBD9
:103AA000B24723A00700B24791073E85EFC09FAB06
:103AB000B2473E85F24005618280397106DE2AC632
:103AC0002EC432C236C0B2473ED402D21247B70724
:103AD00000FFF98F81C77370043001A0924781E71E
:103AE0007370043001A0EFF0EF94AA8799E3824746
:103AF00099E3854711A0814781E77370043001A0E5
:103B0000EFE04FABA2579C433ED0A24532458524FF
:103B10000257A2475D8F9247F98F12476310F70251
:103B20000257A247D98F3ED6A2579843924793C7D0
:103B3000F7FF7D8FA25798C302C025A0824799CF77
:103B4000A257938647001247B7070005D98F024650
:103B5000BE853685EFE03F8902D621A0A2579C435F
:103B60003ED6EFE0EFA62ACE8247B1CBF24799E3EB
:103B7000EFC0DF89EFF06FAF2AD63257B7070002E8
:103B8000F98F85EBEFF08FA7A2579C433ED63257B3
:103B90009247F98F1247631AF700A257984392474A
:103BA00093C7F7FF7D8FA25798C3EFF00FA8854703
:103BB0003ED23257B7070001FD17F98F3ED6B257F4
:103BC0003E85F250216182805D7186C62ACE2ECC60
:103BD00032CA36C83AC6F2473EDA02DC02D8F247A9
:103BE00081E77370043001A06247B70700FFF98FC7
:103BF00081C77370043001A0E24781E7737004301D
:103C000001A0EFF02F83AA8799E3B24799E3854794
:103C100011A0814781E77370043001A0EFE08F9914
:103C2000D2579C433ED64246E245325575242AD4AB
:103C3000A25799CFB2573EDE02C6D247A9CBD25780
:103C40009843E24793C7F7FF7D8FD25798C381A06F
:103C5000B24781E7B2573EDE1DA8D24791C76257EF
:103C6000B7070001D98F3EDCC24791C76257B7073B
:103C70000004D98F3EDCD257938647006247E25753
:103C8000D98F3246BE853685EFE0EFF502DEEFE0F4
:103C90002F942AD2B247B9CB925799E3EFC00FF7CE
:103CA000EFF0AF9C2ADE7257B7070002F98F8DEB59
:103CB000EFF0CF94D2579C433EDE4246E245725528
:103CC000212CAA8799CBD24789CBD2579843E24778
:103CD00093C7F7FF7D8FD25798C3EFF00F9502D8A7
:103CE0007257B7070001FD17F98F3EDEF2573E8588
:103CF000B64061618280797106D62AC62EC4B24769
:103D00003ECEB24781E77370043001A02247B70767
:103D100000FFF98F81C77370043001A0EFF00F8EA0
:103D2000F2479C433ECCF2479843A24793C7F7FF24
:103D30007D8FF24798C3EFF04F8FE2473E85B25038
:103D400045618280797106D62AC6B2473ECEEFC061
:103D5000CFF9AA873ECCF2479C433ECAE2473E8554
:103D6000EFC0AFF7D2473E85B250456182805D71AA
:103D700086C62AC62EC402DCB2473ED802DAB24753
:103D800081E77370043001A02247B70700FFF98F65
:103D900081C77370043001A0C25791073ED6B25755
:103DA000A1073ED4EFE00F81B257DC473EDEC25799
:103DB0009843A2475D8FC25798C3BDA8F257DC4312
:103DC0003ED2F2579C433ED002DA0257B70700FFBB
:103DD000F98F3ECE0257B7070001FD17F98F3ED08D
:103DE0007247B7070004F98F89EBC257984382578F
:103DF000F98F89CF85473EDA11A8C2579843825779
:103E0000F98F02576314F70085473EDAD2579DC3F6
:103E10007247B7070001F98F89C762578257D98F58
:103E20003EDCC2579843B7070002D98FBE85725552
:103E3000EFE00FF992573EDE7257A257E310F7F802
:103E4000C2579843E25793C7F7FF7D8FC25798C375
:103E5000EFD01FF8C2579C433E85B6406161828017
:103E6000797106D62AC6B2473ECEF24791073ECCBC
:103E7000EFD05FF40DA0E247D847E247A1076315F2
:103E8000F7007370043001A0E247DC47B705000279
:103E90003E85EFE0EFF2E2479C43F1FF7245752A61
:103EA000EFD01FF30100B25045618280011106CEB0
:103EB0002AC62EC4A24532455D3D0100F24005618F
:103EC0008280011106CE2AC62EC4A2453245253570
:103ED0000100F2400561828001112AC62EC432C25F
:103EE00002CE924781EB3247A247F98F81CF8547B7
:103EF0003ECE09A83247A247F98F22476314F70044
:103F000085473ECEF2473E850561828001112AC673
:103F1000B2473ECCB24799E302CE21A0E2479C4F84
:103F20003ECEF2473E8505618280397106DE2AC6A3
:103F300002D2EFD03FE8975703009387E76E9C4388
:103F400081EB5522975703009387076E054798C367
:103F5000B24789CFA1473E87B247BA973EC6B2471C
:103F60008D8B89C7B247F19B91073EC6B247F9CB0B
:103F70003247E567ED1763E7E70C97570300938730
:103F8000A7693ED497570300938707699C433ED6A1
:103F900031A0B2573ED4B2579C433ED6B257DC4311
:103FA000324763F5E700B2579C43E5F7325797571E
:103FB00003009387E7666307F708A2579C432147EE
:103FC000BA973ED2B2579843A25798C3B257D84334
:103FD000B247B307F740214706076378F704325723
:103FE000B247BA973ECEB257D843B2471D8FF24779
:103FF000D8C3B2573247D8C3F247DC433ECC9757B9
:104000000300938767613ED021A082579C433ED036
:1040100082579C43DC436247E3E9E7FE82579843BB
:10402000F24798C38257724798C397C70100938796
:10403000E73B9843B257DC431D8F97C70100938736
:10404000E73A98C3EFD0DFD8925799E3EF001037E3
:1040500092573E85F25021618280797106D62AC638
:10406000B2473ECCB247BDC3A147B307F040624759
:10407000BA973ECCE2473ECAEFD0DFD3D247DC430B
:104080003EC897570300938727593ECE21A0F24799
:104090009C433ECEF2479C43DC434247E3E9E7FEC4
:1040A000F2479843D24798C3F247524798C3D24742
:1040B000D84397C70100938767339C433E9797C7C0
:1040C00001009387A73298C3EFD09FD00100B25070
:1040D0004561828097C70100938747319C433E85A5
:1040E000828001008280411197C7010093870753A6
:1040F000F19B3EC69757030093870752324798C3F8
:10410000975703009387475123A20700975703004F
:104110009387075165677117D8C397570300938733
:10412000275023A00700B2473EC4A2476567711716
:10413000D8C3A247175703001307874E98C301003F
:104140004101828001112AC62EC432C2A2473ECE4E
:10415000B2473ECC3247A247D98F8D8BA1E319A835
:10416000F2479843E24798C3E24791073ECCF247B3
:1041700091073ECE9247F5173247BA976247E361FF
:10418000F7FE29A87247930717003ECEE2479386B1
:10419000170036CC034707002380E70032479247D9
:1041A000BA976247E360F7FEB2473E8505618280B9
:1041B00001112AC62EC432C232479247D98F8D8B45
:1041C0009DEFA24793F7F70F3ECAD247A207524787
:1041D000D98F3ECAD247C2075247D98F3ECAB2478B
:1041E0003ECE39A0F247138747003ACE524798C3D4
:1041F00032479247BA977247E366F7FE1DA0B2476F
:104200003ECC11A8E247138717003ACC2247137718
:10421000F70F2380E70032479247BA976247E3637C
:10422000F7FEB2473E850561828001112AC6B2477A
:104230003ECE21A0F24785073ECEF24783C7070056
:10424000F5FB7247B247B307F7403E8505618280B0
:1042500001112AC62EC4B247138717003AC683C776
:104260000700A30FF100A247138717003AC483C7C2
:104270000700230FF1008347F10199C70347F101BC
:104280008347E101E309F7FC0347F1018347E101BB
:10429000B307F7403E850561828001112AC62EC40E
:1042A000B2473ECE01002247930717003EC4F247B3
:1042B0009386170036CE034707002380E70083C7A5
:1042C0000700F5F3B2473E850561828001112AC6D9
:1042D00002CE02CC21A0B24785073EC6B24703C733
:1042E000070093070002E308F7FEB24703C7070081
:1042F0009307D0026309F700B24703C7070093078B
:10430000B0026311F704B24783C70700938737FDF4
:1043100093B7170093F7F70F3ECCB24785073EC619
:1043200015A07247BA878A07BA9786073ECEB2476A
:10433000138717003AC683C70700938707FD7247A4
:10434000BA973ECEB24783C70700E1FFE24789C76D
:10435000F247B307F04011A0F2473E850561828025
:1043600001112AC6975703009387C72D9C43938654
:104370001700175703001307E72C14C332471377AE
:10438000F70F975603009386E62FB6972380E70032
:104390003247A947630BF700975703009387872A93
:1043A0009843930700046315F70497570300938716
:1043B000672D3ECE05A8F247138717003ACE03C7F4
:1043C0000700B70710F0938707F098C397570300CB
:1043D000938747279C431387F7FF975703009387DB
:1043E000672698C3975703009387C7259C43E1F737
:1043F00081473E85056182804D7123261114232457
:1044000081142322911423202115232E3113232CD0
:104410004113232A51132ACE2ECC32C836CA3AC6AB
:104420003EC442C223260112B2473E8A814AC24795
:1044300052485286D6863E85C285EF10205FAA87F5
:104440002E883E86C2868327C11213871700232633
:10445000E11232878A07141AB69723AEE7EEB24705
:104460003E848144D247268763E8E702D247268705
:104470006396E700C247228763E0E702B2473E89BE
:1044800081494A86CE864245D245EF00707CAA8794
:104490002E883EC842CA49BF010029A0F247E24522
:1044A00012458297A2471387F7FF3AC40327C11228
:1044B000E346F7FE25A88327C1128A07181ABA9780
:1044C00003A7C7EF8327C1128A07141AB69783A6DA
:1044D000C7EFA54763F5D7009307700519A09307A9
:1044E0000003BA977247E2453E8502978327C112BF
:1044F0001387F7FF2326E112E34FF0FA0100832030
:10450000C114032481148324411403290114832931
:10451000C113032A8113832A4113716182804111DF
:104520002AC62EC4A2460547635ED700B2479C4305
:104530009D07E19B93868700324714C303A8470079
:104540009C4335A0224719CB324718431306470036
:10455000B24690C21843BA87014811A8324718439F
:1045600013064700B24690C21843BA8701483E85F9
:10457000C2854101828041112AC62EC4A246054748
:10458000635ED700B2479C439D07E19B93868700FB
:10459000324714C303A847009C4305A8224701CF14
:1045A0003247184313064700B24690C21843BA87F1
:1045B0007D873A8819A83247184313064700B24648
:1045C00090C21843BA877D873A883E85C2854101EB
:1045D0008280397106DE22DC26DA2AC62EC432C277
:1045E00036C011A863070424924785073EC2B2472C
:1045F000A24522858297924783C707003E8493078E
:104600005002E311F4FE924785073EC292473EC82E
:1046100093070002A30BF100FD573ECEFD573ECCA1
:1046200002D09247138717003AC283C707003E841F
:104630009307D4FD130750056364F71E13972700F3
:1046400097C70100938707A3BA97984397C70100BC
:10465000938747A2BA9782879307D002A30BF100F2
:10466000C9B793070003A30BF10065BF02CC6247F3
:10467000BA878A07BA978607A297938707FD3ECC29
:10468000924783C707003E849307F00263D68702F0
:104690009307900363C28702924785073EC2C1BF5A
:1046A0008247138747003AC09C433ECC39A0F2476B
:1046B000E3D907F602CEB5B70100F247E3D307F618
:1046C000E2473ECEFD573ECCA9BF825785073ED07C
:1046D00089BF8247138747003AC09C433247A245AF
:1046E0003E850297B1A28247138747003AC08443B0
:1046F00089E497C4010093846497F2476357F004F8
:10470000034771019307D0026301F704E247BE85B6
:104710002685EF00B0512A87F247998F3ECE11A827
:10472000834771013247A2453E850297F247FD1744
:104730003ECEF247E346F0FE09A8B247A2452285E5
:1047400082978504F247FD173ECE83C704003E845E
:104750001DC0E247E3C307FEE247FD173ECCE24738
:10476000E3DD07FC09A8B247A245130500028297C2
:10477000F247FD173ECEF247E347F0FE55A88A8781
:1047800082553E85CD3BAA872E883ED442D6A2577D
:104790003258C28763D90702B247A2451305D00237
:1047A0008297A255325681470148B386B740368575
:1047B00033B5A7003307C840B307A7403E87B68785
:1047C0003A883ED442D6A9473ED21DA8A9473ED238
:1047D00015A0A1473ED239A885473ED0B247A24591
:1047E000130500038297B247A245130580078297FD
:1047F000C1473ED28A8782553E8515332AD42ED6AC
:104800001257834771013E88F2472256B256A2459D
:104810003245DD3631A8B247A2452285829709A8E4
:10482000B247A245130550028297C2473EC201001B
:10483000D9B30100F2506254D254216182804111F7
:104840002AC6B70710F0938707F2324798C301A032
:104850005D7106D62AC62EDA32DC36DEBAC0BEC29A
:10486000C2C4C6C69C0891173ECEF247BE863246E9
:104870008145170500001305E5AEA13B81473E8544
:10488000B2506161828001112AC62EC41EC2A247A5
:104890003ECEF2479C4332471377F70F2380E70061
:1048A000F2479C4313871700F24798C30100056144
:1048B00082801D7106DE2AC62EC4B2C4B6C6BAC82E
:1048C000BECAC2CCC6CE9C103ED25C084C081706AD
:1048D0000000130686FB7D779346F7FF05651305F9
:1048E00005803388A5003378E8001368783B23A05F
:1048F00007013295698F13677733D8C333F7D50033
:104900009315470137870300130737394D8F98C731
:104910003377D6009316470137070300130777064E
:10492000558FD8C70F100000B2473ED69C10A11774
:104930003ED422575C083E857C00BA862246BE855E
:104940004939B24723800700B2473E87B257B307C1
:10495000F7403E85F250256182804111370510F005
:10496000130545F408412AC6370510F0130505F470
:1049700008412AC4370510F0130545F40841B24830
:10498000E39EA8FC32452A83814313170300814626
:104990002245AA850146B3E7B6003368C70037074A
:1049A00010F0130587F48565938505FA0146B386F3
:1049B000B700B688B3B8F8003307C800B387E8007B
:1049C0003E87B6873A881CC12322050101004101B8
:1049D0008280411106C651379307000873A0473003
:1049E0000100B24041018280011106CE2AC617B5EE
:1049F00001001305A57DEFF0BFE50100F240056160
:104A00008280011106CE2AC617B501001305857CE8
:104A1000EFF01FE40100F24005618280797106D653
:104A20002AC602CE29A00100F24785073ECE724772
:104A3000856793877738E3D8E7FE17B5010013053C
:104A4000E579EFF0FFE0F1BF797106D62AC602CE14
:104A500029A0F121F24785073ECE7247CD47E3DA20
:104A6000E7FE0100B25045618280011106CE952219
:104A700017070000130787FD8146054693052003AD
:104A800017B5010013050576EFE07F9E2AC6EFD02B
:104A9000EFC8AA87014781463E8685453245EFE04B
:104AA0003FA30100F24005618280011106CE02C6DB
:104AB000592A2A878547630CF70017B501001305AB
:104AC000E572EFF0FFD8B24793E727003EC6B24742
:104AD0003E85F24005618280011106CE02C6713723
:104AE0001707000013076704814605469305400633
:104AF00017B5010013050571EFE07F972AC6B2478D
:104B000099CBEFD0AFC1AA87014781463E86854544
:104B10003245EFE0FF9B02C4EFD0EF9F81473E8517
:104B2000F24005618280797106D62AC697C70100D6
:104B30009387C78A9C431387470697C701009387CB
:104B4000E78998C397C70100938787899C43138798
:104B5000470697C701009387A78898C397C70100A6
:104B60009387C78798439307F07C63D3E70497C77D
:104B700001009387A7869C431387078397C701008B
:104B80009387C78598C315372ACEF24799EB97C705
:104B900001009387E784984385679387F77663DB03
:104BA000E700F2473E85EFF09FC9EFD0AF9E21A00E
:104BB000010011A00100B250456182807370043081
:104BC00001A00100828041112AC62EC473700430F6
:104BD00001A0411106C681480148975703009387F9
:104BE00067B7054781461306004097B501009385D6
:104BF0002562170500001305A512EFC05F8B9757BC
:104C00000300938727B594438148014897570300D1
:104C1000938787B405471306004097B50100938535
:104C2000A55F170500001305E525EFC05F889757BE
:104C30000300938727B29C433E85EFC03FE5010008
:104C4000B24041018280411185473EC6975703001B
:104C50009387C7A9984397570300938767A89C43F6
:104C60006313F70002C697570300938767A798431B
:104C700097570300938787A798C302C4B9A0175713
:104C800003001307E7A6A2478A07BA9798439756E7
:104C900003009386E6A3A2478A07B6979C43631353
:104CA000F70002C617570300130787A2A2478A0717
:104CB000BA97984397560300938686A3A2478A071C
:104CC000B69798C3A24785073EC422478947E3D8D1
:104CD000E7FA97B701009387E77198438547630325
:104CE000F70002C697B7010093870771984397575B
:104CF00003009387A7A09C436314F70002C619A87A
:104D000097B701009387476F98439757030093879E
:104D1000E79E98C3B2473E8541018280797106D6ED
:104D20002AC602CA5C083E85F525712DAA878D45E5
:104D30003E85EF10E026AA873ECE175703001307E3
:104D40006798F2478A07BA979C433ECC17570300EF
:104D500013070798F2478A07BA979C4313871700EF
:104D6000975603009386C696F2478A07B69798C36C
:104D70005C0881467D56BE856245EFB03FBF2A87FD
:104D800085476308F70097B701009387A76623A0BC
:104D90000700D24785073ECA5247C167FD17631314
:104DA000F70002CA112051B7411106C697570300F8
:104DB000938707959C4313871700975703009387A2
:104DC000279498C397570300938787939843C547C1
:104DD00063F4E70A975703009387879223A007009D
:104DE00097570300938707929C4305476389E7021F
:104DF000054763E6E7000947638CE704B5A89757C2
:104E00000300938767959C4381453E85EFC0BFB300
:104E1000975703009387078F054798C3B1A8975703
:104E20000300938767939C4385453E85EFC0BFB1E0
:104E300097570300938707929C4381453E85EFC0B7
:104E40009FB0975703009387E78B094798C32DA01E
:104E500097570300938707909C4385453E85EFC095
:104E60009FAE975703009387E78923A00700130598
:104E7000800CEFC0FF9601000100B240410182802A
:104E8000797106D62AC6892E0145EFC01FA5AA87CB
:104E900099E302CE19A0FD573ECE975703009387A2
:104EA000E7839C43FD553E85EFC0AFD42ACCE24753
:104EB00091EBF247F1DB97B701009387A75323A04B
:104EC0000700D9B75C0881460146BE856245EFB050
:104ED0009FDC2A8785476308F70097B7010093870F
:104EE000675123A00700EFD07FF1D2473E855920BC
:104EF000EFD0BFF397B701009387C74F984385471B
:104F0000E314F7F8974703009387877D9C43138743
:104F10001700974703009387A77C98C3B5B7411143
:104F200006C6974703009387E77B98438547631F2F
:104F3000F702974703009387277D9C431387170049
:104F4000974703009387477C98C39747030093874D
:104F5000A77B98439307400663FAE700974703004F
:104F60009387877A23A007005122E9220100B240EB
:104F700041018280011106CE2AC63247C167F91766
:104F800063F2E7083247C17785073E97954763F894
:104F9000E7023247E15763E4E70297B701009387DE
:104FA000E7459C43BE853245E5202A87854763084F
:104FB000F70097B701009387E74323A0070097B74F
:104FC0000100938727439C4381E77370043001A05D
:104FD00097B70100938787429C431387170097B7C1
:104FE00001009387A74198C397B7010093870741B2
:104FF0009C43D9EB97B701009387474041677D17E2
:1050000098C359A03247954763FCE702C1671387ED
:10501000E7FFB2471D8F994763F4E7029747030004
:105020009387C76E9C43BE8532459D202A8785475E
:105030006308F70097B701009387C73B23A00700D9
:1050400097B701009387073B9C4381E77370043057
:1050500001A0974703009387676B9C431387170052
:10506000974703009387876A98C3974703009387FE
:10507000E7699843C167F91763F8E70097470300AA
:105080009387C76823A007000100F2400561828072
:1050900001112AC62EC485473ECE3247A24763F38C
:1050A000E7023247A2471D8F8D4763F5E700737013
:1050B000043001A03247A2471D8F8D4763F4E702F9
:1050C00002CE0DA02247B2471D8F8D4763F5E70042
:1050D0007370043001A02247B2471D8F8D4763F3E0
:1050E000E70002CEF2473E8505618280011106CEBF
:1050F000974703009387875E9C433E85EFC06FB15F
:105100002AC6B24785C73C000146BE853245EFB08E
:10511000FFD02A8785476308F70097B70100938778
:10512000672D23A00700A2473E85A9350100F24064
:1051300005618280411106C6974703009387475D4A
:105140009C43174703001307E7578A07BA979C4306
:105150008146014697B501009385052A3E85EFB04B
:105160007F982A8785476315F70697B701009387CD
:10517000A7289C431387170097B701009387C72779
:1051800098C397B70100938727279C4381EB97B774
:1051900001009387672641677D1798C397470300EF
:1051A000938707579C4313871700974703009387FC
:1051B000275698C397470300938787559843894795
:1051C00063D8E700974703009387875423A007001D
:1051D0000100B24041018280011106CE02C4254582
:1051E000EFC0EF972A87974703009387274F98C30D
:1051F00002C65DA0014691450D45EFB0CFD5AA8608
:10520000174703001307074CB2478A07BA9794C39E
:10521000174703001307074BB2478A07BA979C4307
:1052200081E77370043001A0174703001307874913
:10523000B2478A07BA979843974703009387074A6C
:105240009C43BE853A85EFC04F932A878547630903
:10525000F70097B701009387E71923A0070015A867
:105260001747030013070746B2478A07BA979843C0
:1052700097470300938787469C43BE853A85EFC0D6
:10528000CF8FAA8799C797B701009387A71623A046
:105290000700B24785073EC632478947E3DCE7F49B
:1052A00097470300938707429C4381453E85EFC0A3
:1052B0004F90AA8799C797B701009387A71323A098
:1052C0000700974703009387E73F984397470300FA
:1052D0009387C7409C43BE853A85EFC08F8D2A8750
:1052E00085476308F70097B701009387A71023A0AD
:1052F0000700974703009387E73C9C4338008146AB
:105300000146BA853E85EFB06FE697470300938765
:10531000673B9843974703009387473C9C43BE8570
:105320003A85EFC08F85AA8799C797B70100938701
:10533000670C23A00700974703009387A7389C4377
:10534000380081460146BA853E85EFB0DF94974725
:1053500003009387273798439747030093870738BD
:105360009C43BE853A85EFC04F812A8785476308F5
:10537000F70097B701009387E70723A00700974737
:1053800003009387A7359C439305800C3E85EFC0AF
:105390004F86AA8799C797B701009387A70523A0CF
:1053A0000700974703009387E73A9C433E85EFC089
:1053B0001F80974703009387E732054798C3010092
:1053C000F24005618280411106C69747030093872A
:1053D000A7319843B757C6419385D7E63A85EF0082
:1053E000F034AA873E878D67938797033E97974748
:1053F00003009387672F98C3974703009387C72EAF
:105400009C4313D70701A167FD17F98F3E85B24072
:105410004101828041112AC6974703009387C72C18
:10542000324798C30100410182800000B305B500F6
:10543000930705006386B70003C7070063160700DC
:105440003385A74067800000938717006FF09FFEA9
:10545000130101FD23229102232A51012326110267
:105460002324810223202103232E3101232C4101F7
:105470002328610123267101232481012322910124
:105480002320A101930A050093840500639E06383A
:10549000130406009309050017B90100130949D840
:1054A00063F8C512B7070100138B05006378F61087
:1054B0001307F00F3337C70013173700B357E60051
:1054C0003309F900834609003387E600930600029A
:1054D000B386E640638C0600B394D40033D7EA0069
:1054E0003314D600336B9700B399DA00935A040152
:1054F00093850A0013050B00EF00902A130905009D
:1055000093850A00931B040113050B00EF00D024C0
:1055100093DB0B01930405009305050013850B0035
:10552000EF00D0201319090193D70901B367F900DF
:10553000138A040063FEA700B3878700138AF4FF71
:1055400063E8870063F6A700138AE4FFB387870048
:10555000B384A74093850A0013850400EF0050240C
:105560001309050093850A0013850400EF00D01E7F
:105570009399090193040500930505001319090186
:1055800013850B0093D90901EF00501AB369390153
:105590001386040063FCA900B30934011386F4FFE9
:1055A00063E6890063F4A9001386E4FF13140A017B
:1055B0003364C400130A00006F000013B707000132
:1055C00013070001E36CF6EE130780016FF01FEF85
:1055D000138A0600631A06009305000013051000E5
:1055E000EF00901713040500B7070100637EF41263
:1055F0009307F00F63F48700130A8000B357440148
:105600003309F900034709009306000233074701F5
:10561000B386E64063940612B3848440130A1000F4
:10562000135B040193050B0013850400EF00501772
:105630001309050093050B0013850400931B040157
:10564000EF00901193DB0B01930405009305050017
:1056500013850B00EF00900D1319090193D7090171
:10566000B367F900938A040063FEA700B38787003D
:10567000938AF4FF63E8870063F6A700938AE4FF48
:10568000B3878700B384A74093050B0013850400FC
:10569000EF0010111309050093050B00138504009A
:1056A000EF00900B93990901930405009305050001
:1056B0001319090113850B0093D90901EF00100795
:1056C000B36939011386040063FCA900B3093401EE
:1056D0001386F4FF63E6890063F4A9001386E4FFF0
:1056E00013940A013364C4001305040093050A00EF
:1056F0008320C10203248102832441020329010281
:105700008329C101032A8101832A4101032B01015D
:10571000832BC100032C8100832C4100032D010049
:105720001301010367800000B7070001130A00019D
:10573000E366F4EC130A80016FF05FEC3314D400DD
:1057400033DAE400B399DA0033D7EA00935A04015C
:10575000B394D40093850A0013050A00336B9700B5
:10576000EF0010041309050093850A0013050A00D1
:10577000931B0401EF00407E93DB0B0193040500B3
:105780009305050013850B00EF00407A13190901FA
:1057900013570B013367E900138A0400637EA700E7
:1057A00033078700138AF4FF636887006376A700D6
:1057B000138AE4FF33078700B304A74093850A00E8
:1057C00013850400EF00C07D1309050093850A00CE
:1057D00013850400EF00407893040500930505004D
:1057E00013850B00EF00807413170B01135707018B
:1057F00013190901B367E9001387040063FEA700CA
:10580000B38787001387F4FF63E8870063F6A70078
:105810001387E4FFB3878700131A0A01B384A740F4
:10582000336AEA006FF0DFDF63ECD51EB7070100D3
:1058300063F4F6041307F00FB335D70093953500E2
:1058400033D7B60097B701009387879DB387E700EA
:1058500003C70700130A00023307B700330AEA4000
:1058600063160A0213041000E3E096E833B6CA0098
:10587000134416006FF05FE7B707000193050001BE
:10588000E3E0F6FC930580016FF09FFBB35CE6005C
:10589000B3964601B3ECDC0033D4E40093DB0C0197
:1058A000B397440133D7EA0093850B001305040036
:1058B000336BF700B3194601EF00806E1309050042
:1058C00093850B0013050400139C0C01EF00C068C6
:1058D000135C0C01930405009305050013050C00EF
:1058E000EF00C0641319090113570B013367E90076
:1058F00013840400637EA700330797011384F4FF29
:10590000636897016376A7001384E4FF3307970168
:10591000B304A74093850B0013850400EF00406893
:105920001309050093850B0013850400EF00C06286
:10593000930405009305050013050C00EF00005FBC
:1059400093170B011319090193D70701B367F900E6
:105950001386040063FEA700B38797011386F4FF44
:1059600063E8970163F6A7001386E4FFB387970106
:1059700013140401B70B01003364C4001389FBFF47
:10598000337D240133F92901B384A740930509002D
:1059900013050D00EF008059935C04019305090085
:1059A000130B050013850C00EF00405893D9090133
:1059B000130C05009385090013850C00EF000057B8
:1059C000130905009385090013050D00EF0000562B
:1059D0003305850193570B013385A7006374850157
:1059E0003309790193570501B387270163E6F40270
:1059F000E392F4BCB70701009387F7FF3375F50016
:105A000013150501337BFB0033964A01330565010D
:105A1000130A0000E37AA6CC1304F4FF6FF09FB9D9
:105A2000130A0000130400006FF01FCC130101FBE8
:105A30002324810423229104232E31032322910362
:105A40002326110423202105232C4103232A51035B
:105A50002328610323267103232481032320A10328
:105A6000232EB101930C0500938905001304050052
:105A700093840500639E062613090600138A060018
:105A800097AA0100938ACA7963F4C514B707010085
:105A90006376F6129307F00F63F4C700130A8000D1
:105AA000B3574601B38AFA0003C70A001305000280
:105AB00033074701330AE540630C0A00B3954901F7
:105AC00033D7EC0033194601B364B70033944C016B
:105AD000935A090193850A0013850400EF00404C96
:105AE0009309050093850A00131B0901138504001F
:105AF000EF008046135B0B019305050013050B00B7
:105B0000EF00C0429399090193570401B3E7F900EC
:105B100063FAA700B387270163E6270163F4A700B0
:105B2000B3872701B384A74093850A001385040037
:105B3000EF0000479309050093850A0013850400D0
:105B4000EF008041131404019305050093990901A6
:105B500013050B0013540401EF00403D33E48900AA
:105B6000637AA40033042401636624016374A400EF
:105B7000330424013304A440335544019305000049
:105B80008320C104032481048324410403290104E4
:105B90008329C103032A8103832A4103032B0103C1
:105BA000832BC102032C8102832C4102032D0102AD
:105BB000832DC1011301010567800000B7070001B3
:105BC000130A0001E36EF6EC130A80016FF05FED3B
:105BD000631A06009305000013051000EF00C0379C
:105BE00013090500B7070100637AF90E9307F00F58
:105BF00063F42701130A8000B3574901B38AFA00FE
:105C000003C70A0013050002B38429413307470183
:105C1000330AE540E30E0AEA33194901B3DAE90031
:105C2000B395490133D7EC0093540901336BB700A6
:105C300013850A0093850400EF0080369309050060
:105C400093850400931B090113850A00EF00C030FF
:105C500093DB0B019305050013850B00EF00002D6E
:105C60009399090193570B01B3E7F90033944C0161
:105C700063FAA700B387270163E6270163F4A7004F
:105C8000B3872701B38AA7409385040013850A00D0
:105C9000EF000031930905009385040013850A0085
:105CA000EF00802B9305050013850B00EF00002803
:105CB00093150B019399090193D50501B3E5B9003B
:105CC00063FAA500B385250163E6250163F4A50009
:105CD000B3852501B384A5406FF09FDFB7070001AE
:105CE000130A0001E36AF9F0130A80016FF0DFF094
:105CF000E3E8D5E8B707010063FCF604930BF00F67
:105D000033B5DB001315350033D7A60097A7010084
:105D100093870751B387E70083CB07009305000201
:105D2000B38BAB00338B7541631E0B0263E436010A
:105D300063EACC003384CC40B386D94033B58C00C1
:105D4000B384A64013050400938504006FF05FE35D
:105D5000B707000113050001E3E8F6FA1305800117
:105D60006FF09FFAB3966601335D7601336DDD0007
:105D700033D47901B395690133DC7C0193540D016F
:105D8000336CBC001305040093850400B31A66014C
:105D9000EF000021130A0500938504001305040099
:105DA00033996C01931C0D01EF00001B93DC0C0177
:105DB000130405009305050013850C00EF00001780
:105DC000131A0A0113570C013367EA00130A04007F
:105DD000637EA7003307A701130AF4FF6368A701D6
:105DE0006376A700130AE4FF3307A701B309A740AE
:105DF0009385040013850900EF00801A9385040041
:105E00001304050013850900EF0000159305050034
:105E10009304050013850C00EF00401193150C014D
:105E20001314040193D50501B365B400138704006E
:105E300063FEA500B385A5011387F4FF63E8A50100
:105E400063F6A5001387E4FFB385A501131A0A01C1
:105E5000B70C0100336AEA001384FCFFB3778A00B1
:105E600033F48A00B384A54013850700930504002A
:105E70002326F100135A0A01EF00400B9309050095
:105E80009305040013050A00EF00400A13DC0A0121
:105E9000930D050093050C0013050A00EF0000099F
:105EA0008327C100130A050093050C001385070022
:105EB000EF00C0073305B50113D709013307A70069
:105EC0006374B701330A9A01B70701009387F7FF9C
:105ED000935507013377F70013170701B3F7F9005C
:105EE000B3854501B307F70063E6B400639EB400D1
:105EF000637CF90033865741B3B7C700B385A5412A
:105F0000B385F54093070600B307F9403339F9002C
:105F1000B385B440B385254133947501B3D7670188
:105F20003365F400B3D565016FF09FC51306050016
:105F30001305000093F61500638406003305C500C1
:105F400093D5150013161600E39605FE6780000032
:105F50006340050663C60506138605009305050024
:105F60001305F0FF630C060293061000637AB60077
:105F70006358C0001316160093961600E36AB6FE27
:105F80001305000063E6C500B385C5403365D50041
:105F900093D6160013561600E39606FE678000009F
:105FA00093820000EFF05FFB13850500678002001D
:105FB0003305A04063D80500B305B0406FF0DFF9AA
:105FC000B305B04093820000EFF01FF93305A04005
:105FD000678002009382000063CA0500634C0500DD
:105FE000EFF09FF71385050067800200B305B0400E
:105FF000E35805FE3305A040EFF01FF63305B0402F
:0460000067800200B3
:02000004800278
:1000000049444C45000000001C31FEFFE430FEFF77
:10001000F230FEFF0031FEFF0831FEFF2C32FEFF02
:10002000F431FEFF0232FEFF1032FEFF1832FEFFF7
:10003000546D722053766300B037FEFFB037FEFF79
:10004000B037FEFF2E38FEFFFE37FEFF2438FEFFDE
:10005000B037FEFFB037FEFF2E38FEFFFE37FEFF43
:10006000546D725100000000286E756C6C29000000
:10007000B245FEFFB047FEFFA647FEFFB047FEFFBA
:10008000B047FEFFB047FEFFB047FEFF3046FEFF21
:10009000B047FEFFB047FEFFE845FEFF3E46FEFFCD
:1000A000B047FEFFF245FEFFFC45FEFFFC45FEFFAC
:1000B000FC45FEFFFC45FEFFFC45FEFFFC45FEFF48
:1000C000FC45FEFFFC45FEFFFC45FEFFB047FEFF82
:1000D000B047FEFFB047FEFFB047FEFFB047FEFF50
:1000E000B047FEFFB047FEFFB047FEFFB047FEFF40
:1000F000B047FEFFB047FEFFB047FEFFB047FEFF30
:10010000B047FEFFB047FEFFB047FEFFB047FEFF1F
:10011000B047FEFFB047FEFFB047FEFFB047FEFF0F
:10012000B047FEFFB047FEFFB047FEFFB047FEFFFF
:10013000B047FEFFB047FEFFB047FEFFB047FEFFEF
:10014000B047FEFFB047FEFFB047FEFFB047FEFFDF
:10015000B047FEFFB047FEFFB047FEFFB047FEFFCF
:10016000B047FEFFB047FEFFB047FEFFB047FEFFBF
:100170006246FEFF0E47FEFFB047FEFFB047FEFFA0
:10018000B047FEFFB047FEFFB047FEFFB047FEFF9F
:10019000B047FEFF5A46FEFFB047FEFFB047FEFFE6
:1001A0006247FEFF6847FEFFB047FEFFB047FEFF15
:1001B0007646FEFFB047FEFF5C47FEFFB047FEFFFE
:1001C000B047FEFF8047FEFF6D69616F750A000052
:1001D0006D69616F75320A0068756E6772790A0021
:1001E00054696D65723200004572726F7220696EDB
:1001F00020787878207461736B73200D0A000000FA
:10020000436865636B54696D65720000536574548F
:10021000780000005365745278000000000102026B
:10022000030303030404040404040404050505058E
:10023000050505050505050505050505060606066A
:10024000060606060606060606060606060606064E
:10025000060606060606060606060606070707073A
:10026000070707070707070707070707070707071E
:10027000070707070707070707070707070707070E
:1002800007070707070707070707070707070707FE
:1002900007070707070707070707070708080808EA
:1002A00008080808080808080808080808080808CE
:1002B00008080808080808080808080808080808BE
:1002C00008080808080808080808080808080808AE
:1002D000080808080808080808080808080808089E
:1002E000080808080808080808080808080808088E
:1002F000080808080808080808080808080808087E
:10030000080808080808080808080808080808086D
:0C03100008080808080808080808080881
:10031C001000000000000000017A5200017C010175
:10032C001B0D02004C000000180000001851FEFFCD
:10033C00DC05000000440E307089039507810188AC
:10034C000292049305940696089709980A990B9AB9
:10035C000C0370020AC144C844C944D244D344D4E7
:10036C0044D544D644D744D844D944DA440E004446
:10037C000B0000005000000068000000A456FEFFB7
:10038C000005000000440E507488028903930599FF
:10039C000B810192049406950796089709980A9A7E
:1003AC000C9B0D0320010AC144C844C944D244D358
:1003BC0044D444D544D644D744D844D944DA44DB55
:0803CC00440E00440B00000088
:1003E000AAAAAAAA08000000FC8F010009000000C8
:0C03F00001000000FFFF0000FFFF000004
:040000058000004037
:00000001FF
